:100000000C9463000C948B000C948B000C944F07A1
:100010000C944F070C944F070C948B000C948B009E
:100020000C948B000C948B000C948B000C948B0024
:100030000C948B000C948B000C948B000C948B0014
:100040000C9405070C948B000C94D3060C94AD060D
:100050000C948B000C948B000C948B000C948B00F4
:100060000C948B000C948B000000000024002700EF
:100070002A0000000008000201000003040700003D
:1000800000000000000000000000230026002900FE
:1000900000000000250028002B00040404040404D0
:1000A0000404020202020202030303030303010227
:1000B00004081020408001020408102001020408F6
:1000C0001020F507870B11241FBECFEFD8E0DEBF4D
:1000D000CDBF11E0A0E0B1E0E4E5FAE102C0059097
:1000E0000D92AA39B107D9F722E0AAE9B1E001C01F
:1000F0001D92AC3FB207E1F710E0C2E6D0E004C0C9
:100100002197FE010E94ED0BC136D107C9F70E946D
:10011000D4080C941D0D0C9400001092F70250911D
:10012000D602E5EDF2E090E030E020E0591729F04A
:100130004191240F311D9F5FF9CF9091DB024091D7
:10014000DC026091D70270E07093CC026093CB0226
:100150006091D9027091DA0276276727762770932B
:10016000CE026093CD02882379F081E090E09093F5
:10017000CC028093CB02E091C902F091CA02309781
:10018000D9F08BEC92E009945091D5028091A402B1
:10019000581719F082E090E0EACF892F90E0982F6D
:1001A0008827840F911D3195219531098217930776
:1001B00011F383E090E0DBCF0895AF92BF92CF922E
:1001C000DF92EF92FF920F931F93CF93DF936C0117
:1001D0007B018B01040F151FEB015E01AE18BF08F8
:1001E000C017D10759F06991D601ED91FC910190AA
:1001F000F081E02DC6010995892B79F7C501DF91C2
:10020000CF911F910F91FF90EF90DF90CF90BF9013
:10021000AF900895FC01538D448D252F30E0842F3D
:1002200090E0821B930B541710F0CF96089501971E
:100230000895FC01918D828D981761F0A28DAE0F0B
:10024000BF2FB11D5D968C91928D9F5F9F73928F92
:1002500090E008958FEF9FEF0895FC01918D828DBE
:10026000981731F0828DE80FF11D858D90E008958B
:100270008FEF9FEF0895FC01918D228D892F90E0E3
:10028000805C9F4F821B91098F739927089580E0AE
:1002900092E00E943B0121E0892B09F420E0822FAB
:1002A000089580E090E0892B29F00E944701811198
:1002B0000C9400000895FC01A48DA80FB92FB11D66
:1002C000A35ABF4F2C91848D90E001968F7399278C
:1002D000848FA689B7892C93A089B1898C9183706A
:1002E00080648C93938D848D981306C00288F38963
:1002F000E02D80818F7D80830895EF92FF920F9390
:100300001F93CF93DF93EC0181E0888F9B8D8C8DC1
:1003100098131AC0E889F989808185FF15C09FB7B5
:10032000F894EE89FF896083E889F9898081837078
:10033000806480839FBF81E090E0DF91CF911F9127
:100340000F91FF90EF900895F62E0B8D10E00F5F48
:100350001F4F0F731127E02E8C8D8E110CC00FB61E
:1003600007FCFACFE889F989808185FFF5CFCE01B6
:100370000E945B01F1CFEB8DEC0FFD2FF11DE35AD5
:10038000FF4FF0829FB7F8940B8FEA89FB89808139
:100390008062CFCFCF93DF93EC01888D8823B9F0B3
:1003A000AA89BB89E889F9898C9185FD03C0808180
:1003B00086FD0DC00FB607FCF7CF8C9185FFF2CFFD
:1003C000808185FFEDCFCE010E945B01E9CFDF91F7
:1003D000CF910895833081F028F4813099F08230F4
:1003E000A9F008958730A9F08830C9F08430B1F4BD
:1003F000809180008F7D03C0809180008F778093F3
:100400008000089584B58F7784BD089584B58F7D6D
:10041000FBCF8091B0008F778093B00008958091DA
:10042000B0008F7DF9CFCF93DF9390E0FC01E255D0
:10043000FF4F249186569F4FFC0184918823C9F079
:1004400090E0880F991FFC01E859FF4FA591B491E6
:10045000FC01E057FF4FC591D49161110DC09FB7CA
:10046000F8948C91209582238C938881282328836B
:100470009FBFDF91CF910895623051F49FB7F894F8
:100480003C91822F809583238C93E8812E2BEFCF94
:100490008FB7F894EC912E2B2C938FBFEACF3FB7F8
:1004A000F8948091DF019091E001A091E101B09179
:1004B000E20126B5A89B05C02F3F19F00196A11DAA
:1004C000B11D3FBFBA2FA92F982F8827BC01CD019E
:1004D000620F711D811D911D42E0660F771F881FFD
:1004E000991F4A95D1F708952FB7F8946091DB01D1
:1004F0007091DC018091DD019091DE012FBF0895A4
:100500000F931F93CF938C01C0E0D8015D968C911F
:100510005D97C81788F45E968C9160E0811101C0E8
:1005200062E0D8015B96ED91FC91EC0FF11D8081AA
:100530000E941302CF5FE9CFCF911F910F910895D1
:10054000FC01442321F013861486168615868485C3
:10055000258536852115310541F02130310579F0A9
:1005600061112DC0168615860895811106C0662377
:1005700021F021E030E03687258764870895838560
:10058000982F929596959770891B662319F0895F2D
:10059000838703C0811110C01386938589EF890F6B
:1005A000813D60F081E0983D08F480E0138622E010
:1005B00030E03687258708958150EACF80E008959E
:1005C0008F929F92AF92BF92CF92DF92EF92FF9263
:1005D0000F931F93CF93DF93EC01A12CF12CE12C0F
:1005E0000FEF1FEF8D8DA81608F039C0CA2CD12C43
:1005F000EB8DFC8DEC0DFD1D208130E0F901EE58F6
:10060000FF4F8491F901E255FF4FB490F901E6568E
:10061000FF4F9490992001F181110E94EA01E92D88
:10062000F0E0EE0FFF1FEA57FF4FA591B491EC9158
:10063000BE2231E020E009F430E0832F922F2E8D8E
:100640002817190639F40F3F100709F48601EFEF58
:10065000EE1AFE0AA394C6CF90E080E0F0CF60E0EF
:10066000EA94EF28F1F4888D998D8017910749F06D
:1006700041E060E0CE010E94A0021B821A821D822E
:100680001C8261E0888D998D8017910709F060E0E8
:10069000198F088F8B8D9C8D080F191FF801808191
:1006A0008F8B40E0CE010E94A002F82E0C811D81AC
:1006B0000115110581F01D821C82C801DF91CF91C7
:1006C0001F910F91FF90EF90DF90CF90BF90AF9070
:1006D0009F908F9008958A819B818230910509F4C3
:1006E000C2C040F40097A1F1019709F441C0F11094
:1006F000E4CF87C08430910509F47DC008F4DFC0E1
:100700000597A9F7FF2009F47CC00E947402CE80EF
:10071000DF80E884F984AB01BC014C195D096E09E6
:100720007F098D899E89B0E0A0E0481759076A07C4
:100730007B0718F28A8506E010E083FD02C003E023
:1007400010E00E9474026E837F8388879987B5CFFB
:10075000FF2009F4B2CF81E090E09B838A830E945E
:1007600074026E837F838887998701E010E0A5CFAC
:10077000F1100FC08A8582FF30C082E090E09B8339
:100780008A830E9474026E837F838887998702E040
:1007900010E00E947402CE80DF80E884F984AB010F
:1007A000BC014C195D096E097F098F859889B0E0FD
:1007B000A0E084179507A607B70708F07ECF0E9430
:1007C00074026E837F83888799878A8581FF0CC036
:1007D00084E090E09B838A8370CF83E090E09D83E8
:1007E0008C831B821A82D3CF80FF66C085E090E0A5
:1007F0009B838A832EC0F11009C085E090E09D8321
:100800008C831B821A8202E010E057CF0E94740290
:10081000CE80DF80E884F984AB01BC014C195D090E
:100820006E097F098B899C89B0E0A0E08417950749
:10083000A607B70708F041CF8A8580FF0DC085E085
:1008400090E09B838A830E9474026E837F838887F3
:10085000998703E010E031CF86E090E09B838A83A4
:1008600005E010E02ACFFF2061F083E090E09B8359
:100870008A830E9474026E837F838887998701E050
:1008800010E00E9474028E809F80A884B984AB011E
:10089000BC01481959096A097B0989899A89B0E01C
:1008A000A0E084179507A607B70708F006CF90E0E9
:1008B00080E0FF2009F49CCF86E090E099CFF11012
:1008C00008C084E090E09D838C831B821A8202E042
:1008D00010E00E9474028E809F80A884B984AB01CE
:1008E000BC01481959096A097B098F859889880FC5
:1008F000991FB0E0A0E0481759076A077B0708F482
:10090000DCCE83E090E09D838C8386E090E0F11064
:1009100061CF90E080E05ECF2091E5013091E6016B
:100920002817390771F49091E3018091E401981739
:1009300041F0E091E301F0E0E656FE4F808190E067
:1009400008958FEF9FEF08950895EF92FF920F9310
:100950001F93CF93DF93DC015C96ED90FC905D9745
:10096000E114F10479F481E090E013969C938E9366
:10097000129790E080E0DF91CF911F910F91FF904F
:10098000EF9008955196ED91FC91529750968C916D
:100990005097982F90950FB75E962C915E97122FD7
:1009A000127021FD6095F8942081112319F1282BF4
:1009B0002083E7012197F1F728E0462F50E03081AE
:1009C00060FF1AC0382B3083E7012197F1F7BA0195
:1009D00075956795215089F7112381F080818923CE
:1009E00080830FBF5C968D919C910197F1F781E018
:1009F00090E0C1CF2923DCCF3923E5CF9081892B2B
:100A0000EFCF2091E5013091E6012817390771F405
:100A10008091E4012091E30190E0805C9F4F821B74
:100A2000910960E470E00E94A30B089590E080E0DB
:100A300008952091E5013091E60128173907B9F4AE
:100A40009091E3018091E401981789F0E091E3012E
:100A5000F0E0E656FE4F80812091E30130E02F5F09
:100A60003F4F2F7333272093E30190E008958FEFDA
:100A70009FEF08950F931F93CF93DF93C091F702D9
:100A8000CC2321F10E9474020091F3021091F40230
:100A90002091F5023091F602601B710B820B930BD3
:100AA0000091D0021091D1022091D2023091D30254
:100AB000601771078207930748F081E00E948D005C
:100AC0008C2FDF91CF911F910F9108958AEA92E0C8
:100AD0000E940105892B79F11DE18AEA92E00E94CA
:100AE0001905C82F8091A302C81302C01092F20208
:100AF000E091F20281E08E0F8093F202F0E0E35683
:100B0000FD4FC7AB8E3110F01093F2028AEA92E0EB
:100B10000E9401052091A902892B79F0D22FC213DE
:100B2000DCCF2D1303C080E00E948D00C1E08091D6
:100B3000A9028D1729F2C0E0C3CFDC2FF2CF8F922C
:100B40009F92AF92BF92CF92DF92EF92FF929091DD
:100B5000F80191111DC09091A3029093EE01909124
:100B6000A4029093EF019091A5029093F0019091CF
:100B7000A7029093F2019091A8029093F5019093AF
:100B8000F6019091A9029093F70191E09093F801FA
:100B90008093F1016093F3014093F4014091F001DF
:100BA000EFEEF1E020E090E080E0421729F0319193
:100BB000830F911D2F5FF9CF9195819591099093A6
:100BC000F5018093F6014AE050E06EEE71E08AEAAA
:100BD00092E00E94DD000E944F024B015C0184E123
:100BE000C82ED12CE12CF12C0E944F0268197909F2
:100BF0008A099B09683E734081059105A8F321E0AD
:100C0000C21AD108E108F10888EE880E83E0981E28
:100C1000A11CB11CC114D104E104F10429F70E9404
:100C200074026093F3027093F4028093F502909340
:100C3000F6021092CC021092CB0281E08093F70270
:100C40008091CF02882321F00E943A058823E1F3A6
:100C5000FF90EF90DF90CF90BF90AF909F908F90DC
:100C60000895462F682F8FE090E00C949F0590E048
:100C700080E00895CF93DF93CDE9D2E04091000169
:100C80006B858EE490E00E949F0588A9DF91CF914B
:100C90000895FC0187890895FC0101900020E9F77F
:100CA0003197AF01481B590BBC0180E092E00C94D6
:100CB000DD008F929F92AF92BF920F931F93CF93BD
:100CC000DF93CDB7DEB7A1970FB6F894DEBF0FBEA6
:100CD000CDBF19A2423008F44AE08E010F5D1F4FCC
:100CE000842E912CB12CA12CA50194010E94B70B4C
:100CF000E62FB901CA01EA30F4F4E05DD801EE93C1
:100D00008D01232B242B252B79F790E080E0109781
:100D100019F0CD010E944C06A1960FB6F894DEBFE3
:100D20000FBECDBFDF91CF911F910F91BF90AF90BC
:100D30009F908F900895E95CE1CFCF93DF930E945D
:100D40004C06EC0181E491E00E944C068C0F9D1F43
:100D5000DF91CF9108950E94180D1F920F920FB648
:100D60000F9211242F933F934F935F936F937F9331
:100D70008F939F93AF93BF93EF93FF9380E092E0A5
:100D80000E945B01FF91EF91BF91AF919F918F9175
:100D90007F916F915F914F913F912F910F900FBE77
:100DA0000F901F9018951F920F920FB60F9211245B
:100DB0002F938F939F93EF93FF93E0911002F09105
:100DC00011028081E0911602F091170282FD1BC092
:100DD0009081809119028F5F8F7320911A02821780
:100DE00041F0E0911902F0E0E050FE4F958F8093C2
:100DF0001902FF91EF919F918F912F910F900FBE4C
:100E00000F901F9018958081F4CF1F920F920FB60C
:100E10000F9211242F933F938F939F93AF93BF9380
:100E20008091DB019091DC01A091DD01B091DE01A8
:100E30003091DA0123E0230F2D3758F50196A11DDB
:100E4000B11D2093DA018093DB019093DC01A09324
:100E5000DD01B093DE018091DF019091E001A0916E
:100E6000E101B091E2010196A11DB11D8093DF0166
:100E70009093E001A093E101B093E201BF91AF91A3
:100E80009F918F913F912F910F900FBE0F901F90C8
:100E9000189526E8230F0296A11DB11DD2CF1F92EF
:100EA0000F920FB60F9211242F933F934F935F939E
:100EB0006F937F938F939F93AF93BF93EF93FF9322
:100EC000E091E501F091E601309749F0A685B785FC
:100ED0008585968D91FF14C09C918923A1F4FF9183
:100EE000EF91BF91AF919F918F917F916F915F91A2
:100EF0004F913F912F910F900FBE0F901F9018951B
:100F00009C91892361F7A389B4899C9185898095F7
:100F100089238C93868997890197F1F7608D718D6C
:100F2000A685B785558538E020E0CB010197F1F71C
:100F3000822F90E095958795282F4C91452309F0B5
:100F40002068315091F7868D81FD20958091E401D4
:100F500090E001968F7399273091E301381799F04B
:100F6000A091E401B0E0A656BE4F2C938093E4011B
:100F7000828D938D0197F1F7A389B4898C9195891E
:100F8000892B8C93ACCF868D8160868FF1CF1F9398
:100F9000CF93DF93282F30E0F901EE58FF4F849173
:100FA000F901E255FF4FD491F901E656FF4FC49184
:100FB000CC23A9F0162F81110E94EA01EC2FF0E05A
:100FC000EE0FFF1FE057FF4FA591B4918FB7F89434
:100FD000EC91111108C0D095DE23DC938FBFDF9117
:100FE000CF911F910895DE2BF8CF1092030210923B
:100FF000020288EE93E0A0E0B0E0809304029093B8
:101000000502A0930602B093070221E231E030937B
:1010100001022093000225EC30E030930D02209372
:101020000C0224EC30E030930F0220930E0220ECEF
:1010300030E0309311022093100221EC30E0309325
:1010400013022093120222EC30E030931502209319
:10105000140226EC30E0309317022093160210920F
:10106000190210921A0210921B0210921C022EE119
:1010700020939D0210929E0261E060939F02609314
:10108000A00222E02093A10224E02093A2022EE7F6
:101090002093A3022FEF2093A40226E02093A50221
:1010A0001092A6026093A7021092A8022FEE20933E
:1010B000A9021092AD021092AC028093AE029093FE
:1010C000AF02A093B002B093B10283E391E090939A
:1010D000AB028093AA021092C1021092C002109239
:1010E000C3021092C2021092C5021092C402109262
:1010F000C7021092C6028091C8028E7F8D7F8093B6
:10110000C80286958170682786E00E94C70761E063
:1011100086E00E941302E4EBF0E0E491E093BA026F
:10112000E0EAF0E0E491F0E0EE0FFF1FE057FF4F40
:10113000859194919093BC028093BB0260E085E01E
:101140000E9413028091C80281FD04C061E085E025
:101150000E94C70785E08093B602E3EBF0E0E491DC
:10116000E093B702EFE9F0E0E491F0E0EE0FFF1F4B
:10117000EA57FF4F859194919093B9028093B802FA
:101180001092CA021092C90281E08093CF0288EEC9
:1011900093E0A0E0B0E08093D0029093D102A093BE
:1011A000D202B093D3020895CF93DF9300D000D042
:1011B0001F92CDB7DEB7789484B5826084BD84B5C4
:1011C000816084BD85B5826085BD85B5816085BD42
:1011D00080916E00816080936E00109281008091FA
:1011E0008100826080938100809181008160809382
:1011F0008100809180008160809380008091B100A7
:1012000084608093B1008091B00081608093B000D1
:1012100080917A00846080937A0080917A00826065
:1012200080937A0080917A00816080937A00809127
:101230007A00806880937A001092C100E0911002D9
:10124000F091110282E08083E0910C02F0910D0296
:101250001082E0910E02F0910F028FEC80831092C9
:101260001802E0911402F091150286E08083E0916B
:101270001202F0911302808180618083E09112025A
:10128000F0911302808188608083E0911202F091D6
:101290001302808180688083E0911202F091130232
:1012A00080818F7D808360E082E00E94130260E095
:1012B00083E00E94130242E06091A80289E090E07E
:1012C0000E949F05C090D002D090D102E090D2023F
:1012D000F090D3021092C5021092C4021092C30281
:1012E0001092C2021092C1021092C0028DE991E0E8
:1012F0009093C7028093C6029091B602963108F08F
:1013000047C02DEB30E03093C1022093C0022BE99F
:1013100031E03093C3022093C2022CE231E03093DB
:10132000C5022093C4022091680084E0983048F000
:1013300031E09E3008F430E081E001C0880F3A953A
:10134000EAF7822B809368002DE630E0983050F069
:101350002BE630E09E3030F02CE630E0963110F095
:1013600030E020E03093BE022093BD02292F30E010
:10137000983008F028C181E001C0880F9A95EAF7FB
:101380008093BF028091C6029091C7020197F1F746
:101390008091C4029091C502892B49F1E091E50149
:1013A000F091E60122E0EA3AF20709F1309739F0CC
:1013B000A389B4899C918589809589238C93809198
:1013C000C8028E7F8093C8021092E4011092E3015C
:1013D0008AEA92E09093E6018093E501E091BD02F4
:1013E000F091BE0280819091BF02892B808380EDB5
:1013F00097E0A0E0B0E08093D0029093D102A09358
:10140000D202B093D3026091A802462F8CE090E004
:101410000E949F05C092D002D092D102E092D202E7
:10142000F092D3024091A1026091A80289E090E07D
:101430000E949F050E9474026B017C010E943A0584
:1014400081110BC00E9474026C197D098E099F09DD
:10145000683E73408105910588F381E08093CF0257
:101460000E943A0540919D02493108F049E160919E
:10147000A80286E090E00E949F056091A802462F96
:101480008FE490E00E949F058091CD02815080936F
:10149000E7010E943A068093E801EBE1F1E0FA836C
:1014A000E9830AEE11E09BE0A92E91E0B92ECC244D
:1014B000CA94DC2C34EFE32EFF24F39442E5642E2F
:1014C00043E0742E58EB452E5BE0552E60E1262E4E
:1014D00067E2362E75E1872E71E0972E8FE190E05E
:1014E0000E94F30B9D838C83A981BA81ED91BA830D
:1014F000A983EB83DC011196BC92AE9213961C92E9
:101500001E9212971B961C921B975996DC92CE92B4
:1015100058975096FC92EE921F9752967C926E923C
:1015200051971A968C911A9754965C924E925397B3
:1015300056963C922E925597877F87601A968C9389
:101540001A9741E060E0CD010E94A002EC81FD818C
:101550001382128215821482918280822B81228FC3
:10156000CF014A96948F838F81E0858F868FD80133
:10157000ED93FD938D01CF010E948002E981FA81F4
:10158000ED51F14009F0AACF80E0E82E80E0F82E7E
:101590000E943A050AEE11E01982D8018D919D91C1
:1015A0008D01DC01ED91FC910280F381E02D099524
:1015B0000097E1F183309105F9F090F40197B0F5CF
:1015C0008EE891E016C09E3040F42850310981E049
:1015D00001C0880F2A95EAF7D3CE2E503109F7CFF4
:1015E0008530910509F451C080F1069749F781E8EB
:1015F00091E00E944C061AC084E491E00E949D068E
:10160000B981BB23B9F18091E9019091E801891773
:1016100020F48F5F8093E90103C0E1E0E093E901EA
:101620006091E901809100010E943106F981F13059
:1016300039F5E114F10409F4ABCF0E944701882386
:1016400009F4A6CF0E940000A3CF8EE491E00E948F
:101650009D068091E901F981FF2341F09091E80115
:101660008917B8F221E02093E901DACF815059F0CF
:101670008093E9016091E901809100010E943106A7
:1016800081E089838ACF81E0F3CF89E591E00E94F0
:101690009D0699819923B9F1809100019091E7010C
:1016A000891758F5A1E0A093E9018F5F80930001AD
:1016B0000E943A068093E80187E691E00E944C067A
:1016C0006091E80170E090E080E04AE00E945906F5
:1016D00081E491E00E944C0682E791E00E944C0672
:1016E0006091000170E090E080E04AE00E945906BD
:1016F00081E491E00E944C0693CFB1E0B093E90100
:10170000B0930001D9CFE1E0E093E901D5CF83E3C5
:1017100091E09093AB028093AA028091E5019091B1
:10172000E6018A5A924071F4E091BD02F091BE0246
:1017300090818091BF028095892380831092E60179
:101740001092E501089597FB072E16F4009407D038
:1017500077FD09D00E94D90B07FC05D03EF4909587
:1017600081959F4F0895709561957F4F0895A1E2EF
:101770001A2EAA1BBB1BFD010DC0AA1FBB1FEE1F0B
:10178000FF1FA217B307E407F50720F0A21BB30B56
:10179000E40BF50B661F771F881F991F1A9469F7D2
:1017A00060957095809590959B01AC01BD01CF012E
:1017B0000895AA1BBB1B51E107C0AA1FBB1FA61798
:1017C000B70710F0A61BB70B881F991F5A95A9F7EA
:1017D00080959095BC01CD010895EE0FFF1F0590F7
:1017E000F491E02D09940F931F93CF93DF938230F0
:1017F000910510F482E090E0E091FA02F091FB0292
:1018000030E020E0B0E0A0E0309799F421153105F8
:1018100009F44AC0281B390B24303105D8F58A81D8
:101820009B816115710589F1FB0193838283FE0120
:1018300011C0408151810281138148175907E0F09E
:101840004817590799F4109761F012960C93129764
:1018500013961C933296CF01DF91CF911F910F9178
:1018600008950093FA021093FB02F4CF211531057D
:1018700051F04217530738F0A901DB019A01BD016D
:10188000DF01F801C1CFEF01F9CF9093FB02809304
:10189000FA02CDCFFE01E20FF31F81939193225004
:1018A000310939832883D7CF2091F8023091F9028A
:1018B000232B41F420910301309104013093F9026C
:1018C0002093F80220910101309102012115310588
:1018D00041F42DB73EB74091050150910601241BFC
:1018E000350BE091F802F091F902E217F307A0F44A
:1018F0002E1B3F0B2817390778F0AC014E5F5F4F66
:101900002417350748F04E0F5F1F5093F90240939C
:10191000F802819391939FCFF0E0E0E09CCFCF93CA
:10192000DF930097E9F0FC01329713821282A091B5
:10193000FA02B091FB02ED0130E020E01097A1F433
:1019400020813181820F931F2091F8023091F9029A
:101950002817390709F061C0F093F902E093F80203
:10196000DF91CF910895EA01CE17DF07E8F54A81AC
:101970005B819E0141155105B1F7E901FB83EA83C3
:1019800049915991C40FD51FEC17FD0761F480816F
:1019900091810296840F951FE90199838883828142
:1019A00093819B838A83F0E0E0E012968D919C9175
:1019B00013970097B9F52D913C911197CD0102969F
:1019C000820F931F2091F8023091F90228173907EE
:1019D00039F6309751F51092FB021092FA02B0934B
:1019E000F902A093F802BCCFD383C2834081518116
:1019F000840F951FC817D90761F44E5F5F4F888128
:101A00009981480F591F518340838A819B81938319
:101A100082832115310509F0B0CFF093FB02E093EA
:101A2000FA029ECFFD01DC01C0CF13821282D7CF14
:101A300081E090E0F8940C941D0D10E0C2E6D0E037
:101A400004C0FE010E94ED0B2196C336D107C9F7F1
:041A5000F894FFCF38
:101A5400010000FC02800000000000AB06AB064958
:101A640006000000008002E00249060203000000B4
:101A7400007D01DD000A01CA013B0119012D0100AD
:101A8400000000A504DD003706A404010519058C37
:101A9400040D0A004B45595F5052455353004B45C2
:101AA400595F445052455353004B45595F4C4F4E78
:101AB40047505245535300746F74616C736F6E6773
:101AC400200063757272656E74666F6C6465722053
:101AD400004B45595F5250545052455353004B45A7
:0A1AE400595F554E4B4E574E00005F
:00000001FF
